:100000000C9434000C9451000C9451000C94510049
:100010000C9451000C9451000C9451000C94FC0170
:100020000C9451000C9451000C9461010C945100FB
:100030000C9451000C941B010C9451000C94510031
:100040000C9451000C9451000C945F000C945100DE
:100050000C946D000C9451000C9451000C945100C0
:100060000C9451000C94510011241FBECFEFD8E026
:10007000DEBFCDBF11E0A0E0B1E0E6E2F6E002C0F5
:1000800005900D92A433B107D9F711E0A4E3B1E0D4
:1000900001C01D92AD34B107E1F70E946C020C94CF
:1000A00011030C9400001092C00088ED8093C100F1
:1000B0001092C5008CE08093C400789408951F923C
:1000C0000F920FB60F9211248F938091C6008F91DB
:1000D0000F900FBE0F901F9018951F920F920FB6A2
:1000E0000F9211248F93EF93FF93E0914A01F091C7
:1000F0004B013196F0934B01E0934A013197809187
:100100004C01815080934C0180914C01882319F05F
:1001100081818093C600FF91EF918F910F900FBE68
:100120000F901F901895CF92DF92FF920F931F931D
:10013000DF93CF93CDB7DEB72C970FB6F894DEBF21
:100140000FBECDBF6C019B0177FD02C0FF2408C02C
:10015000309521953F4F8DE2F6018083FF24F39483
:1001600040E08E010F5F1F4F0FC0E00FF11FC9016C
:100170006AE070E00E94C802805D8083C9016AE085
:1001800070E00E94C8029B01E42FF0E04F5F2A302C
:1001900031055CF70E0F1F1F822F805DF8018083F1
:1001A000442319F480E3898341E0842F90E09E0189
:1001B0002F5F3F4FF901E80FF91F1082DC01119703
:1001C000A20FB31F90E02EE2491729F4F601EF0DBC
:1001D000F11D2083F394F601EF0DF11D8C918083C6
:1001E000F3949F5F1197941778F3F601EF0DF11DCB
:1001F0001082C6012C960FB6F894DEBF0FBECDBF9D
:10020000CF91DF911F910F91FF90DF90CF900895D4
:10021000FC0180914C01882349F4F0934B01E09359
:100220004A0160934C0180818093C60080914C010B
:100230008823E1F708951F920F920FB60F921124B1
:100240008F939F93AF93BF938FEF9FEFA0E0B0E0AA
:1002500080932B0190932C01A0932D01B0932E013C
:1002600010924701109246015D98BF91AF919F9106
:100270008F910F900FBE0F901F901895209810929D
:10028000800083EC8093810010928200EFE6F0E022
:10029000808181628083789408950AC020E030E0F4
:1002A00000002F5F3F4F42E0203D3407C9F7019720
:1002B0000097A1F7089502C0000001970097E1F7A9
:1002C00008951F920F920FB60F9211242F933F9310
:1002D0004F935F936F937F938F939F93AF93BF934E
:1002E000EF93FF93109285001092840080912B0170
:1002F00090912C01A0912D01B0912E0180932F019E
:1003000090933001A0933101B09332018091860027
:1003100090918700A0E0B0E080932B0190932C0196
:10032000A0932D01B0932E011092870010928600A9
:1003300080912F0190913001A0913101B091320153
:100340008F5F9F4FA040B040F9F020912B0130917A
:100350002C0140912D0150912E0160E47DE083E05D
:1003600090E00E94DB02309345012093440180918C
:1003700044019091450144975CF083E190E09093B3
:1003800045018093440104C0109247011092460138
:1003900080914401909145019093470180934601DB
:1003A00080914801882339F4299A81E090E00E94E5
:1003B0004D01299810C0299A80E991E00E945B01C3
:1003C00029981092490184EF8093B3001092B200F3
:1003D00087E08093B100FF91EF91BF91AF919F9122
:1003E0008F917F916F915F914F913F912F910F90DE
:1003F0000FBE0F901F9018951F920F920FB60F927D
:1004000011242F933F934F935F936F937F938F9319
:100410009F93AF93BF93EF93FF93809149018130F6
:1004200049F41092B1005D9A299A88EC90E00E94FC
:100430005B012998809149018F5F80934901FF9169
:10044000EF91BF91AF919F918F917F916F915F914C
:100450004F913F912F910F900FBE0F901F901895C5
:10046000CF93DF93EC0180914C01882381F4D093EA
:100470004B01C0934A01DE010D900020E9F711976E
:10048000AC1BBD0BA0934C0188818093C60080916A
:100490004C018823E1F7DF91CF9108950F931F93CB
:1004A000DF93CF9300D000D00F92CDB7DEB7BC0161
:1004B0008E010F5F1F4FC80140E00E949300C801EA
:1004C0000E9430020F900F900F900F900F90CF91DD
:1004D000DF911F910F9108951F93219A2998559AA2
:1004E0005D980E943E0192E09093B00087E0809377
:1004F000B1008FEF8093B300809170008260809391
:10050000700097BB78941092C00088ED8093C10072
:100510001092C5008CE08093C400789480E091E054
:100520000E94300211E080912B0190912C01A0914A
:100530002D01B0912E018F5F9F4FA040B04019F464
:100540008DE091E015C020912B0130912C0140915C
:100550002D0150912E0160EE70E782E790E00E943D
:10056000DB02C901109348010E944E028BE191E029
:100570000E943002809146019091470190958195AB
:100580009F4F0E944E0283E291E00E943002CBCF47
:1005900097FB092E07260AD077FD04D02ED006D06F
:1005A00000201AF4709561957F4F0895F6F79095A5
:1005B00081959F4F0895A1E21A2EAA1BBB1BFD0136
:1005C0000DC0AA1FBB1FEE1FFF1FA217B307E40732
:1005D000F50720F0A21BB30BE40BF50B661F771F8A
:1005E000881F991F1A9469F760957095809590956A
:1005F0009B01AC01BD01CF010895AA1BBB1B51E1BA
:1006000007C0AA1FBB1FA617B70710F0A61BB70B82
:10061000881F991F5A95A9F780959095BC01CD0127
:060620000895F894FFCFDD
:1006260048616C6C6F20546573740D0A00456E67E3
:10063600696E65204F6666202D20002055706D205E
:100646002D200020477261640D0A00FFFF0000FFA5
:04065600FF000000A1
:00000001FF
